:03010000C31C011C
:10011C002100003922EC020E19CD05003C320301FE
:10012C003A0700672E00F921000022180121010076
:10013C00221A010E0021900111D001CD8A011180EB
:10014C00001A471305FA7B011AFE20CA4F01FE3E26
:10015C00CA0502FE3CCAD801CD8A011305FA780102
:10016C001AFE20C267013E0012C34F013E00120668
:10017C0000C5219001E53E02CD0D0DC3CE027323C7
:04018C0072230CC905
:1001D00050474D4E414D4500CD3202FA5802E5CD13
:1001E0003C02D5C5216702E5216302E5CDEC05D1CE
:1001F000D17CB5CA5802221801C1D1E13EFFB8CA6C
:100200007B01C34F01CD3202FA5802E5CD3C02D545
:10021000C5216702E5216502E5CDEC05D1D17CB5AC
:10022000CA5802221A01C1D1E13EFFB8CA7B01C3FC
:100230004F011305F81AFE20CA3202C9216702C510
:100240000E1077132305FA53020DCA58021AFE2026
:10025000C242023600E14DC91177020E09CD0500F8
:07026000C3CE02720077001B
:10027700696F6C69623A09556E61626C6520746FCB
:10028700206F70656E203C206F72203E2066696C7F
:1002970065243333C1D1E1EDB8E5D5C53B3BC9335F
:1002A70033C1D1E1EDB0E5D5C53B3BC93A0700679E
:1002B7002E00C92ABE02C90000E1D1C1C5D5E5CDCE
:1002C70005006F079F67C92A1A017CB7CADB02E5D9
:1002D700CDC506C13A03015F1D0E0ECD05002AEC00
:1002E70002F9C300000000C1D1D5C5D5210B03E534
:1002F700210200E5CDEB0AC1C1210200CD870BE544
:10030700C1C3CE020D0D41626F727465642C2072F9
:100317006561736F6E203D20000604216D0311A8EF
:10032700003E80BECA37031905C22A03210000C94F
:10033700360011DFFF19C9C1E1E5C51121001936E2
:0503470080210000C947
:03036D008000000D
:0304150080000064
:0304BD00800000BC
:0305650080000013
:1005EC00C1E1220E01D1EB220C01E5D5C5CD2003D2
:1005FC002204017CB5C8112400192206012A060127
:10060C0011040019EB2A0601010000097323722A58
:10061C000401E52A0C01E5CD8907E1E12A04016E0C
:10062C002600E5CD650BE12A0E017EFE72CA41065D
:10063C00FE52C26A060E0F2A0401EBCD0500B7F27A
:10064C005A062A0401E5CD3E03E1210000C92A0621
:10065C000111020019110000732372C3C1062A0E86
:10066C00017EFE77CA7806FE57C2B5060E132A0421
:10067C0001EBCD05000E162A0401EBCD0500B7F2F7
:10068C009A062A0401E5CD3E03E1210000C92A06A1
:10069C0001110200191180007323722A0401112127
:1006AC0000193E01B677C3C1062A0401E5CD3E030D
:1006BC00E1210000C92A0401C9C1E1220401E5C5F8
:1006CC007CB72E00C82101002212012A040111213D
:1006DC0000197EE601CA4B07211A00E52A0401E540
:1006EC00CD9909E1E12A0401112400192206012AFD
:1006FC000601110000195E2356EB2208012A06019F
:10070C0011840019220A012A0801EB2A0A017ABC79
:10071C00DA2707C233077BBDD233072A0801361A02
:10072C0023220801C31307211500E52A0401E5CD96
:10073C00110BD1D17CB7F24B072100002212010E14
:10074C00102A0401EBCD0500B7F25E072100002250
:10075C0012012A0401E5CD3E03E12A1201C9C1D1DF
:10076C00D5C5D5216302E5CDEC05D1D12204010E0E
:10077C0013CD05002A0401E5CD3E03D1C9E1D1C159
:10078C00C5D5E5131A1BFE3AC2A6071AD640131399
:10079C00FE20DAA907D620C3A9073A0301020326D3
:1007AC00202E08CDC5072E03CDC50726002E04CD5F
:1007BC00FD07211000093600C97DB7CAE8071AFEEB
:1007CC002ECAE807FE00CAE807FE61DAE107FE7BE5
:1007DC00D2E107D6200203132DC3C5071AFE2ECA79
:1007EC00F707FE00CAF70713C3E807FE2EC2FD0782
:1007FC00137DB7CA09087C02032DC3FD07C9C1E1EB
:10080C00E5C5E5CD2308D17DE67FFE0DC22208E5C6
:10081C00D5CD2308E1E1C9D1E1E5D57CB7C23208D9
:10082C00CDCE08D1D1C9220401112100197EE602D6
:10083C00CA430821FFFFC92A04011124001922060A
:10084C0001110000195E2356EB2208012A06011142
:10085C000200197E23B6C29208211400E52A040175
:10086C00E5CD110BD1D17CB5CA7B0821FFFFC92A7C
:10087C000601110200191180007323722A0601115E
:10088C000400192208012A0601110200195E2356E0
:10089C001B722B732A080123EB2A060101000009A5
:1008AC007323722A08017EE67FFE1AC2C9082A0445
:1008BC0001112100197EF6027721FFFFC97E6F26F8
:1008CC0000C92A18017CB7CADC08E5CD0A08C1C9E1
:1008DC000E01CD05006F2600E67FFE1AC2EE082140
:1008EC00FFFFFE0DC2FC08E50E021E0ACD0500E15D
:1008FC00C9C1E1E5C5E52A18017CB7CA1709EB2186
:10090C005000E5D5CD4709C1C1C1C9E12208012B71
:10091C005636002B5E364FE5D5EB0E0ACD05002A78
:10092C0008012B5E231600193600D1E173237223C4
:10093C000E021E0ACD05002A0801C93333C1D1E1CC
:10094C00E5D5C53B3B78B7C25C09E5CDFD08C1C90F
:10095C00221601D5D11BD57AB3CA9209E5C5CD0AA9
:10096C0008C17CB7CA8709D12A1601EB7CBAC2929E
:10097C00097DBBC29209210000D1C97DE17723E634
:10098C007FFE0DC260093600D12A1601C9C1D1E122
:10099C00E5D5C57AB7C2C7097BFE01C2B009E5CD62
:1009AC00900AE1C9FE02C2B909CDA50AC9FE04C26A
:1009BC00C409E5CDEE09E1C9C3EA09E5D5CD0F0AB5
:1009CC00D17CB7FAE9097DFE0DC2E709210A00E5E1
:1009DC00D5CD0F0AD1D17CB7FAE909E1C9C121FF04
:1009EC00FFC9C1D1D5C52210010E05CD05003A10A5
:1009FC0001FE0DC2090A1E0A0E05CD05002A1001C2
:100A0C002600C9C1D1E1E5D5C5221001EB220401B4
:100A1C0011240019220601110000195E2356EB2245
:100A2C0008012A0601110200197E23B6C2680A21A8
:100A3C001500E52A0401E5CD110BD1D17CB5CA51C5
:100A4C000A21FFFFC92A0601110200191180007347
:100A5C0023722A0601110400192208012A06011129
:100A6C000200195E23561B722B732A080123EB2AF2
:100A7C000601010000097323723A10012A0801775C
:100A8C0026006FC9C1E1E5C5E52A1A017CB7CAA4E5
:100A9C000AE5CD9909C1C1C9E1221001EB0E02CDC5
:100AAC0005003A1001E67FFE0DC2BF0A1E0A0E02B7
:100ABC00CD05002A10012600C9C1E1E5C5E52A1AB9
:100ACC00017CB7CAD90AE5CDEB0AC1C1C9E17EB731
:100ADC00CAEA0A23E56FCDA50A0000C3D90AC9C129
:100AEC00D1E1E5D5C57E23B7CA0D0BE54F0600C590
:100AFC00D5CD9909D1C17CB7CA090BC1C9E1C3F1E4
:100B0C000A210000C9C1D1E1221401EB220401D554
:100B1C00E5C52A04016E2600E5CD650BE12A04012A
:100B2C001124001911040019EB0E1ACD05002A141A
:100B3C00014D2A0401EBCD0500CD7E0B2212010ED6
:100B4C001A118000CD05002A12017CB5C2610B215F
:100B5C000000C3640B21FFFFC9D1E1E5D57DB4CA08
:100B6C00750BEB1B0E0ECD0500C919C37D0B232392
:100B7C00397E6F079F67C919C38A0B2323397E23DC
:100B8C00666FC9232339545DCD7D0B2B7D12C92390
:100B9C002339545DCD7D0B237D12C919C1D1C57D7F
:100BAC0012C9232339545DCD8A0B2BC3CA0B2323C3
:100BBC0039545DCD8A0B23C3CA0B19C1D1C57D1223
:100BCC00137C12C97DB36F7CB267C97DAB6F7CAAF5
:100BDC0067C97DA36F7CA267C9CD0B0CC82BC9CD8F
:100BEC000B0CC02BC9EBCD0B0CD82BC9CD0B0CC8E7
:100BFC00D82BC9CD0B0CD02BC9CD0B0CD82BC97C49
:100C0C00EE80677AEE80BCC2180C7BBD210100C956
:100C1C00CD360CD02BC9CD360CD82BC9EBCD360C20
:100C2C00D82BC9CD360CC8D82BC97ABCC23D0C7B8D
:100C3C00BD210100C9EB1DF87C177C1F677D1F6F60
:100C4C00C3420CEB1DF829C3500C7B956F7A9C6743
:100C5C00C9CD620C23C97C2F677D2F6FC9444D21F0
:100C6C000000790FD2740C19AF781F47791F4FB061
:100C7C00C8AF7B175F7A1757B3C8C36E0C444D7A55
:100C8C00A8F57AB7FCCA0C78B7FCD20C3E10F5EB81
:100C9C0011000029CDDA0CCAB60CCDE20CFAB60C58
:100CAC007DF6016F7B915F7A9857F13DCABF0CF5C9
:100CBC00C39F0CF1F0CDCA0CEBCDCA0CEBC97A2F4B
:100CCC00577B2F5F13C9782F47792F4F03C97B1799
:100CDC005F7A1757B3C97B917A98C97CB5C2EF0C70
:100CEC002E01C9210000C9EBE14E23462378B1CA7D
:100CFC000C0D7E23BB7E23C2F50CBAC2F50C6069C9
:010D0C00E9FD
:0000000000
